:020000040000FA
:1000000000008A1175280000FF00030E8301B00074
:100010000A08B1008A01B12A820701340034003491
:1000200000340A34003400340034643400340034C2
:100030000034E834033400340034103427340034FE
:100040000034A034863401340034403442340F3458
:10005000003480349634983400340034E134F5347C
:1000600005340034CA349A343B342030B200A40141
:10007000A501A601A7010310AC0DAD0DAE0DAF0D8E
:100080000310A00DA10DA20DA30DA40DA50DA60D8D
:10009000A70D27082B02031D572826082A02031D37
:1000A000572825082902031D572824082802031968
:1000B0005B2803186A282808A4022908031C290FB2
:1000C000A5022A08031C2A0FA6022B08031C2B0FCB
:1000D000A7022C14B20B3B2808008000840AB20B44
:1000E0006D2808008A0034088200831338308400A9
:1000F0003330B20000306D208316910183129F01CE
:1001000083169F010730831299009A018316051008
:100110008312401040088500873012052038920075
:10012000FC30120503389200F930831692008C14CB
:100130000B1783128C103230C200B601831687125F
:100140000712071087100711871148308312C30068
:100150006530C4006C30C5006C30C6006F30C7001D
:100160002030C8005730C9006F30CA007230CB0051
:100170006C30CC006430CD000D298312BA003A08EF
:100180000319080001303A0203190800BA030000FD
:100190003A08BB00BC01D1280000000000000000AC
:1001A000BC0A3C083B02031DCC2808005608DB00B3
:1001B0005708DC00DE01DF01EF2883120313023051
:1001C000A0006130A10000008A11A10BE32800000B
:1001D0008A11A00BE1280000DE0A0319DF0A5E087D
:1001E0005B02A0005F085C022004031DDD280800FC
:1001F0008312BD00F0304105BE000F303D05BF0049
:100200003F083E04C10041088700411641088700AD
:1002100000004112410887000800B701BC29DD0039
:1002200002305D0203191629031C1729DD015D0840
:100230000319003401305D020319403402305D02BD
:100240000319143403305D02031954340800831277
:100250002008B800C11641088700380E0F39B900D0
:100260003908F82083123808F8200430BD28D3005C
:1002700053080F218312D60056085507B700803067
:100280003704DA00C112410887005A0E0F39DB002B
:100290005B08F82083125A08F8200430BD2801308A
:1002A0008312D600C11241088700560E0F39DA00BA
:1002B0005A08F82083125608F8200430BD20B430C4
:1002C000BD28C112410887001930D600D701D620B9
:1002D0000330F82005308312D600D701D620033032
:1002E000F8200A30BD200330F8200430BD20023051
:1002F000F8200430BD2028308312D300C1124108F9
:100300008700530E0F39D5005508F8208312530883
:10031000F8200430BD201C308312D300C1124108E4
:100320008700530E0F39D5005508F8208312530863
:10033000F8200430BD200C308312D300C1124108D4
:100340008700530E0F39D5005508F8208312530843
:10035000F8200430BD2006308312D300C1124108BA
:100360008700530E0F39D5005508F8208312530823
:10037000F8200430BD204F2961219E2A5608DE0056
:100380005708DF005E08E4005F08E500E001D629B9
:100390005B086007840083135C1883170008A000C3
:1003A0005308B400540872208312E00A6008640203
:1003B000A00065082004031DC82908005308DE00BA
:1003C0005408DF005608E0005708E1005808E20032
:1003D0005908E3000930EC29E60060086104620472
:1003E0006304031DF9293030A0005E08B4005F08E3
:1003F00072286A146608803AA0008030200203192F
:10040000032A031C9D2A0310660DE8000310E80D63
:1004100000308A0068080C208312A00001306807B1
:100420000C208312A100023068070C208312A20066
:10043000033068070C208312A30063082302031D06
:100440002B2A62082202031D2B2A61082102031DA8
:100450002B2A6008200203192F2A0318822A03106E
:10046000660DE9000310E90D00308A0069080C20D0
:100470008312A800013069070C208312A900023002
:1004800069070C208312AA00033069070C2083122D
:10049000AB006008A0006108A1006208A200630828
:1004A000A300352083122C08E7000310660DE80036
:1004B0000310E80D00308A0068080C208312A800A1
:1004C000013068070C208312A900023068070C2055
:1004D0008312AA00033068070C208312AB00600867
:1004E000A0006108A1006208A2006308A3003520F3
:1004F00083122408E0002508E1002608E20027080E
:10050000E300832AE701E60367086A1603196A1203
:10051000EA126A1CEA166A136A1EEA1A6A176A1F46
:10052000FA2930306704E8006808A0005E08B400CB
:100530005F08722083126A10FA2908008312CE0124
:10054000CF01D001D1014F2127308312D3000130D8
:10055000D4000B30D600D7014330DB00DC01BE21D4
:10056000C32A8C1CBC2A8C10C2034208031DBC2A5F
:100570003230C2000130B60031088A00300E8300EC
:10058000FF0E7F0E0900831212158B178312360897
:100590000319C62AB601051CCF2AD210D02AD214BC
:1005A0004010D218401440088500D5010130372191
:1005B0008312CE0A0319CF0A0319D00A0319D10AEC
:1005C0002730D3000130D4004E08D6004F08D700A2
:0C05D0005008D8005108D900DE21C62ACE
:02400E00D13FA0
:00000001FF
